:020000040000FA
:100000000002040000000000440E0000440E000046
:10001000440E0000440E0000440E0000440E000098
:10002000440E0000440E0000440E0000440E000088
:10003000440E0000DE02000090020000440E0000AA
:10004000440E0000440E0000440E0000440E000068
:10005000440E0000440E0000440E0000440E000058
:10006000440E0000440E0000440E0000440E000048
:10007000440E0000440E0000440E0000440E000038
:10008000440E0000440E0000440E0000440E000028
:10009000440E0000440E0000440E0000440E000018
:1000A000440E0000440E0000440E0000440E000008
:1000B000440E0000440E0000440E0000440E0000F8
:1000C000440E0000440E0000440E0000440E0000E8
:1000D000440E0000440E0000440E0000440E0000D8
:1000E000440E0000440E0000440E0000440E0000C8
:1000F000440E0000440E0000440E0000440E0000B8
:10010000440E0000440E0000440E0000440E0000A7
:10011000440E0000440E0000440E0000440E000097
:10012000440E0000440E0000440E0000440E000087
:10013000440E0000440E0000440E0000440E000077
:10014000440E0000440E0000440E0000440E000067
:10015000440E0000440E0000440E0000440E000057
:10016000440E0000440E0000440E0000440E000047
:10017000440E0000440E0000440E0000440E000037
:10018000440E0000440E0000440E0000440E000027
:10019000440E0000440E0000440E0000440E000017
:1001A000440E0000440E0000440E0000440E000007
:1001B000440E0000440E0000440E0000440E0000F7
:1001C000440E0000440E0000440E0000440E0000E7
:1001D000440E0000440E0000440E0000440E0000D7
:1001E000440E0000440E0000440E0000440E0000C7
:1001F000440E0000440E0000440E0000440E0000B7
:10020000FFFFFF00FFFFFF00440E0000440E000050
:10021000440E0000440E0000440E0000440E000096
:10022000440E0000440E0000440E0000440E000086
:10023000440E0000DE02000090020000440E0000A8
:10024000440E0000440E0000440E0000440E000066
:10025000440E0000440E0000440E0000440E000056
:10026000440E0000440E0000440E0000440E000046
:10027000440E0000440E0000440E0000440E000036
:10028000440E0000440E0000440E0000440E000026
:10029000440E0000440E0000440E0000440E000016
:1002A000440E0000440E0000440E0000440E000006
:1002B000440E0000440E0000440E0000440E0000F6
:1002C000440E0000440E0000440E0000440E0000E6
:1002D000440E0000440E0000440E0000440E0000D6
:1002E000440E0000440E0000440E0000440E0000C6
:1002F000440E0000440E0000440E0000440E0000B6
:10030000440E0000440E0000440E0000440E0000A5
:10031000440E0000440E0000440E0000440E000095
:10032000440E0000440E0000440E0000440E000085
:10033000440E0000440E0000440E0000440E000075
:10034000440E0000440E0000440E0000440E000065
:10035000440E0000440E0000440E0000440E000055
:10036000440E0000440E0000440E0000440E000045
:10037000440E0000440E0000440E0000440E000035
:10038000440E0000440E0000440E0000440E000025
:10039000440E0000440E0000440E0000440E000015
:1003A000440E0000440E0000440E0000440E000005
:1003B000440E0000440E0000440E0000440E0000F5
:1003C000440E0000440E0000440E0000440E0000E5
:1003D000440E0000440E0000440E0000440E0000D5
:1003E000440E0000440E0000440E0000440E0000C5
:1003F000440E0000440E0000440E0000440E0000B5
:100400008F8B2000807E2200000188000000000009
:100410000C000700A0DD20000100200011000700F3
:10042000000020000000E000020032000000020096
:1004300000000000CE040200000000000040DA00CE
:100440000000FE004440A900000020000000E00081
:100450000300320000002000A00188004440A800F2
:100460000000060091018800800078000000EB0089
:1004700015003700E280400032A0B4009101BA00BC
:10048000E280400032A0B4009102BA00E280400055
:1004900032A0B4000002EB00472BDE00F507B200EB
:1004A000602CE10004003A000059EB008301E900F0
:1004B000FDFF3E00040037006128E100010032002A
:1004C0000082EB00040007001101BA000200E00006
:1004D000E8FF3A00000006003159BA008301E90044
:1004E0000C0032002159BA008301E90008003200F3
:1004F0000400E00003003A00E280400032A0B400B3
:10050000F5FF370011D9BA008301E900FAFF3A007C
:100510008100E800E180400032A0B4000000060045
:1005200000A0FE003400F800881F780008002000BA
:10053000A80188004F0478000400FA00807F2200A0
:10054000000F78008480A90060C8BF000004E000AC
:10055000160032000040EB00204798000E003700E4
:100560002E4090008080FB002E4090000080FB0019
:10057000000040001E004000100178008180400013
:10058000C085200000804000020878002E409000C6
:100590000040E800204798002E409000E14F5000B6
:1005A000EFFF36000040EB0060E8B7000080FA0083
:1005B0003400F9000080FE0000400600809FBE006D
:1005C000821F78003400F80000002000A00188009D
:1005D0000000FA005AC8BF000004E00080003A00A2
:1005E000D04080000000E800D0408800D14080006A
:1005F000E0408000808F5000B20036000000EB0029
:10060000D04088003AC8BF00E14F500071003A0066
:10061000CDC2BF000080FB004600DE000004A20047
:1006200061406000614060006140600061406000C6
:100630004601DD00D12C200091407800F0CBB300C2
:1006400000C0600002407000CDE2B700E0418000D1
:10065000E04188000000E800E041880050C8BF0089
:10066000E14F500097003A00CCC2BF000080FB0071
:100670004200DE000004A2006140600061406000B2
:1006800061406000614060004201DD00C12C20003B
:1006900091407800B0CFB30000C06000024070000D
:1006A000CCE2B700CCC2BF000080FB004200DE00FD
:1006B0000004A20061406000614060006140600091
:1006C000614060004301DD00C12C200091407800B2
:1006D00070CFB30000C0600002407000CCE2B700F1
:1006E000CCC2BF000080FB004400DE000004A2007A
:1006F00061406000614060006140600061406000F6
:100700004401DD00C12C200091407800F0CEB30000
:1007100000C0600002407000CCE2B700CCC2BF0055
:100720000080FB004400DE000004A2006140600085
:100730006140600061406000614060004501DD0093
:10074000C12C200091407800F0CDB30000C06000C3
:1007500002407000CCE2B700CDC2BF000080FB00B9
:100760004400DE000004A2006140600061406000BF
:1007700061406000614060004401DD00D12C200038
:1007800091407800F0CEB30000C0600002407000DD
:10079000CDE2B700CDC2BF000080FB004400DE0008
:1007A0000004A200614060006140600061406000A0
:1007B000614060004501DD00D12C200091407800AF
:1007C000F0CDB30000C0600002407000CDE2B70081
:1007D0003C0037000000EB00E041880039003700A2
:1007E000CBC2BF00624060000004E000160032008F
:1007F0000000EB00D04088000000EB00E0418800E2
:1008000056C8BF000004E0002E003A00A14280005C
:10081000E0408000808F500005003E00CDC2A8005F
:10082000A04280000000E800A042880025003700B8
:10083000CDC2A9000000EB00A042880010C0B300A8
:1008400056E8B7001F003700CBC2BF000044B2001B
:100850000004E0001200320056C8BF000004E000AF
:1008600018003A00A1428000E0408000808F5000D4
:1008700005003E00CDC2A800A04280000000E800B4
:10088000A04288000F003700CDC2A9000000EB0095
:10089000A042880010C0B30056E8B7000900370036
:1008A0000000EB00D04088000000EB00E041880031
:1008B0000000EB00A04288000040EB0056E8B700C3
:1008C000CDC2A9008460A9000080FA003400F900BC
:1008D0004F0178004F00BE00004006000000FA0003
:1008E000C04180000000E0000C003A00CCE2A9000A
:1008F000CCC2A80000E2240001002000D4040700BC
:10090000CCC2A900CBC2BF00614060000080FB00E8
:100910000040880010002000C0418800B0418000E5
:100920000000E800B0418800CCE2A800B14180009E
:1009300000062000808F50000F003600CCE2A90096
:1009400062C8BF008080FB00CBC2BF006140600076
:100950000081FB008180400000802000008040007A
:100960000208780062C8BF000040E80062E8B700F3
:100970000000EB00B041880062C8BF00E74F5000A4
:100980000400360010C0B30062E8B7000000EB00BE
:10099000C04188000080FA00000006000400FA0050
:1009A00090022000303A880044C7BF00F043B200F4
:1009B00001C4B3000140700044E7B7004174200057
:1009C0009140780000CEB30000C0600044E7B7005B
:1009D000FF3FFC001000200031742000820720003F
:1009E000A309200082487800834878008048780076
:1009F00010002000217420006204200073052000F4
:100A00008248780083487800804878000000FC0025
:100A100042C7BF00614060000004E000FCFF3A00F4
:100A2000016C20009140780000CEB30000C060004F
:100A30002041B300C0E6B700116C2000914078005F
:100A400000CEB30000C060003041B300C1E6B70083
:100A5000411820009140780080CFB30000C06000B2
:100A600084E1B700A11820009140780080CFB30046
:100A700000C060008AE1B70040062000100C88002A
:100A800040062000400C8800800C2000000C8800EC
:100A9000800C2000300C8800411820009140780024
:100AA00080CFB30000C060006040B30084E1B700B5
:100AB000A11820009140780080CFB30000C06000F2
:100AC0006040B3008AE1B7008461A9008A61A9008F
:100AD00011E1A9001021A90010C1A90001112000F5
:100AE00091407800F0CCB30000C060000044A0004A
:100AF00010E1B7000000EB0030088800A00F2000D4
:100B00006008880011E1A80005E1A9000421A900FE
:100B100004C1A9004110200091407800F0CCB3003E
:100B200000C0600004E1B7000000EB00000888008E
:100B30007038210010088800510A20009140780088
:100B4000F0C8B30000C060000044A000A5E0B700FA
:100B50008460A9009460A80005E1A800007020004E
:100B6000401688003000200000168800C0FF2100D9
:100B700060198800300020008019880021E3A90056
:100B8000013220009140780000CEB30000C0700018
:100B900020E3B7002043A8002183A90023C3BF009E
:100BA0007F40600023E3B7002343A80031322000D8
:100BB00091407800C0CFB30000C0600023E3B700CD
:100BC000213220009140780030CCB30000C060009A
:100BD0000044A00022E3B70025E3A9005132200021
:100BE0009140780000CEB30000C060000004A00077
:100BF00025E3B70020C0B30024E3B7000000EB00FA
:100C0000901988000138200091407800F0CCB300A2
:100C100000C0600001C2B3000140700080E3B70073
:100C200000302000401C88002138200091407800CE
:100C300000C8B30000C06000D040B30082E3B7003A
:100C4000807F2000201C880030002000501C88007D
:100C500081C3A90081A3A9008183A9008163A900A0
:100C60000138200091407800C0CFB30000C0600080
:100C700080E3B7008480A900610A200091407800D9
:100C800080CFB30000C060006040B300A6E0B700B2
:100C90009480A80081E3A80021E3A80010C0B3005D
:100CA00060E8B7006000B800F041880001428800A9
:100CB0001D0037000000EB00000C88000000EB0076
:100CC000300C8800CDC2A80004FF0700104080004F
:100CD0000000E00009003A00204080000000E00031
:100CE00003003A0010002000204288000500370071
:100CF0000000EB0020428800020037000000EB00FB
:100D00002042880000E2240001002000D0030700F8
:100D1000F04180000142800061004000E080480016
:100D2000F041880001428800F241800003428000C7
:100D3000703E200001002000800F5100818F59007B
:100D4000DCFF360020428000E10F500007023A002D
:100D50006000B800F041880001428800FC013700C3
:100D6000DEFE07000000EB0010428800280037007C
:100D70001042800080004000008020000080400081
:100D8000100078000000E00019003A00007D20000B
:100D900001002000AE0307001042800080004000E8
:100DA0000080200000804000100078000000E0007B
:100DB00009003A00104280000000E800504288001C
:100DC00011428000008B2000808040000040EB003A
:100DD000804878000B00370011428000008B200013
:100DE0008080400010C0B3008048780005003700C4
:100DF00011428000008B20008080400010C0B300B2
:100E000080487800104280000000E800104288000E
:100E100010428000E70F5000D5FF3600B0C8BF0079
:100E20008080FB00B1C8BF000080FB0080804000D4
:100E3000B2C8BF000080FB0080804000B3C8BF0084
:100E40000080FB0080804000B4C8BF000080FB0031
:100E500080804000B5C8BF000080FB00808040005B
:100E6000B6C8BF000080FB0080804000B7C8BF004C
:100E70000080FB0000804000E80F500002003A00B4
:100E800010C0B3004EE8B7004EC8BF00E14F50009D
:100E90003F013A00B0C8BF008080FB00B1C8BF006E
:100EA0000080FB0080804000B2C8BF000080FB00D3
:100EB00080804000B3C8BF000080FB0080804000FD
:100EC000B4C8BF000080FB0080804000B5C8BF00F0
:100ED0000080FB0080804000B6C8BF000080FB009F
:100EE00080804000B7C8BF000080FB000080400049
:100EF000E70F500026013A00604280008000400069
:100F000080892000008040009000780050428000DE
:100F1000808F50001C013A000040EB004EE8B70003
:100F2000604280000000E80060428800604280006B
:100F30008000400080892000008040009000780000
:100F4000B0042000808F500011013A00CC0037001F
:100F5000CDC2BF000080FB004600DE000004A200FE
:100F6000614060006140600061406000614060007D
:100F70004601DD00D12C200091407800F0CBB30079
:100F800000C0600002407000CDE2B70000E2240023
:100F9000010020002E0307004FC8BF000080FB00A7
:100FA000100798001E009000E20F50001B00320056
:100FB0009E009000E28F500004003C001E00900054
:100FC000E10F500008003200400037009E00900002
:100FD000E38F5000240032001E009000E40F500008
:100FE0002E00320039003700102C200001002000B4
:100FF00017030700102C2000010020001403070035
:10100000102C20000100200011030700102C2000EC
:10101000010020000E0307002C00370040B0200024
:10102000010020000A03070040B02000010020005A
:101030000703070040B02000010020000403070060
:1010400040B02000010020000103070040B0200054
:1010500001002000FE02070040B020000100200037
:10106000FB0207001900370090E720000100200074
:10107000F702070090E7200001002000F4020700BB
:1010800090E7200001002000F102070090E7200017
:1010900001002000EE0207000C003700205820005D
:1010A00001002000EA020700205820000100200073
:1010B000E70207002058200001002000E40207009A
:1010C0002058200001002000E1020700304280008B
:1010D0004142800061004000E080480030428800CA
:1010E00041428800324280004342800020032000B9
:1010F00001002000800F5100818F590060003600F0
:10110000CCC2BF000080FB004200DE000004A20051
:1011100061406000614060006140600061406000CB
:101120004201DD00C12C200091407800B0CFB30017
:1011300000C0600002407000CCE2B700CCC2BF002B
:101140000080FB004200DE000004A200614060005D
:101150006140600061406000614060004301DD006B
:10116000C12C20009140780070CFB30000C0600017
:1011700002407000CCE2B700CCC2BF000080FB0090
:101180004400DE000004A200614060006140600095
:1011900061406000614060004401DD00C12C20001E
:1011A00091407800F0CEB30000C0600002407000B3
:1011B000CCE2B700CCC2BF000080FB004400DE00E0
:1011C0000004A20061406000614060006140600076
:1011D000614060004501DD00C12C20009140780095
:1011E000F0CDB30000C0600002407000CCE2B70058
:1011F000CDC2BF000080FB004400DE000004A2005E
:1012000061406000614060006140600061406000DA
:101210004401DD00D12C200091407800F0CEB300D5
:1012200000C0600002407000CDE2B700CDC2BF0038
:101230000080FB004400DE000004A200614060006A
:101240006140600061406000614060004501DD0078
:10125000D12C200091407800F0CDB30000C0600098
:1012600002407000CDE2B7006000B8003042880054
:10127000414288004FC8BF000040E8004FE8B70077
:101280004FC8BF00EF4F500031FF3600CC42A900DD
:10129000CC62A900CC82A900CCA2A900CD82A90071
:1012A000CDA2A900CDC2A900104128005101200003
:1012B0006702070010412800510120006402070066
:1012C0001041280051012000610207001041280050
:1012D000510120005E02070010412800510120004A
:1012E0005B0207001041280051012000580207004E
:1012F0000000370060C8BF000004E000FDFF3A00B6
:1013000010C0B30050E8B700300620001008880075
:10131000F1428000203F2000808F50000300360003
:1013200010C0B3003AE8B70012003700B0418000A7
:101330000000E800B0418800F1428000B041800028
:10134000808F50000B0031003AC8BF008040EB0096
:10135000014F78000004E00002003A0010C0B30022
:10136000004F78001E4078003AE8B7000000EB001C
:10137000B0418800E0428000E040880010C0B30027
:1013800060E8B700DBFF37000000EB006042880038
:10139000304280004142800061004000E08048000F
:1013A000304288004142880032428000434280003F
:1013B0008038210001002000800F5100818F5900EA
:1013C0005D003600CCC2BF000080FB004200DE00A2
:1013D0000004A20061406000614060006140600064
:1013E000614060004201DD00C12C20009140780086
:1013F000B0CFB30000C0600002407000CCE2B70084
:10140000CCC2BF000080FB004300DE000004A2004D
:1014100061406000614060006140600061406000C8
:101420004301DD00C12C20009140780070CFB30053
:1014300000C0600002407000CCE2B700CCC2BF0028
:101440000080FB004400DE000004A2006140600058
:101450006140600061406000614060004401DD0067
:10146000C12C200091407800F0CEB30000C0600095
:1014700002407000CCE2B700CCC2BF000080FB008D
:101480004500DE000004A200614060006140600091
:1014900061406000614060004501DD00C12C20001A
:1014A00091407800F0CDB30000C0600002407000B1
:1014B000CCE2B700CDC2BF000080FB004400DE00DC
:1014C0000004A20061406000614060006140600073
:1014D000614060004401DD00D12C20009140780083
:1014E000F0CEB30000C0600002407000CDE2B70053
:1014F000CDC2BF000080FB004500DE000004A2005A
:1015000061406000614060006140600061406000D7
:101510004501DD00D12C200091407800F0CDB300D2
:1015200000C0600002407000CDE2B7006000B8006B
:101530003042880041428800F04180000142800032
:1015400061004000E0804800F041880001428800CE
:10155000F241800003428000F07B220091002000D5
:10156000800F5100818F5900FDFD3600CDC2A900CA
:10157000DAFC0700004080000000E00008003A00AC
:10158000C012200001002000B101070000408000CF
:101590000000E00003003A00CC42A8000100370040
:1015A000CC42A900104080000000E00008003A0092
:1015B000C012200001002000A5010700104080009B
:1015C0000000E00003003A00CC62A80001003700F0
:1015D000CC62A900404080000000E00008003A0012
:1015E000C012200001002000990107004040800047
:1015F0000000E00003003A00CC82A80001003700A0
:10160000CC82A900504080000000E00008003A00B1
:10161000C0122000010020008D0107005040800012
:101620000000E00003003A00CCA2A800010037004F
:10163000CCA2A900604080000000E00008003A0051
:10164000C0122000010020008101070060408000DE
:101650000000E00003003A00CD82A800010037003E
:10166000CD82A900704080000000E00008003A0030
:10167000C0122000010020007501070070408000AA
:101680000000E00003003A00CDA2A80001003700EE
:10169000CDA2A900304080000000E0000F003A0019
:1016A000304180000000E0000E003A0010002000F1
:1016B0003041880020438000E70F500004003E00C6
:1016C000204380000000E800204388000500370028
:1016D0007000200020438800020037000000EB006B
:1016E00030418800204080000000E0000F003A00F8
:1016F000404180000000E0000E003A001000200091
:1017000040418800204380000000E00004003200D7
:10171000204380000000E9002043880005003700D6
:101720000000EB0020438800020037000000EB00BF
:1017300040418800404080000000E00016003A0070
:1017400011C8BF00E74F400011003E00B0408000CC
:101750000000E800B0408800204380008000400086
:10176000808820000080400090007800B040800019
:10177000808F500008003E0011C8BF000040E80004
:1017800011E8B7000000EB00B0408800020037000D
:10179000A0CFB30011E8B700504080000000E00087
:1017A00016003A0011C8BF000004E000110032002A
:1017B000C04080000000E800C04088002043800056
:1017C0008000400080882000008040009000780069
:1017D000C0408000808F500008003E0011C8BF004C
:1017E0000040E90011E8B7000000EB00C0408800AD
:1017F000020037000040EB0011E8B70070408000A5
:101800000000E00016003A0010C8BF00E74F40009B
:1018100011003E00904080000000E80090408800E9
:10182000204380008000400080882000008040002D
:101830009000780090408000808F500008003E00AB
:1018400010C8BF000040E80010E8B7000000EB003F
:101850009040880002003700A0CFB30010E8B70026
:10186000604080000000E00016003A0010C8BF0091
:101870000004E00011003200A04080000000E800F9
:10188000A040880020438000800040008088200025
:101890000080400090007800A0408000808F5000C1
:1018A00008003E0010C8BF000040E90010E8B70083
:1018B0000000EB00A0408800020037000040EB0071
:1018C00010E8B70020438000E70F50000200360008
:1018D000700020002043880010C8BF000080FB007B
:1018E000000C880011C8BF000080FB00300C88008D
:1018F00060C8BF000004E000FDFF3A005AC8BF0006
:101900000004E00008003A00E1428000C0FF2F0020
:101910000088B900800078000002210000804000AB
:10192000E040880007003700E14280000080EB00C3
:101930000088B9008000780000402000008040004E
:10194000E0408800F0428000C2032000110009003E
:101950000280D800A0418800A041800080004000A3
:1019600060862000008040009000780000418000E8
:10197000808F500005003A002041800020418800FF
:101980000000E80020418800020037000000EB0062
:101990002041880020418000F80F500008003600E8
:1019A000A041800080004000608620000080400050
:1019B00010007800F04088000000EB002041880013
:1019C000A041800080004000608620000080400030
:1019D0001000780000418800CBC2BF006440600066
:1019E0000004E00046003200F04080000000E0000B
:1019F00003003A0010C0B3005AE8B7006A0037008D
:101A00000040EB005AE8B700F1408000A00420003D
:101A1000808F500011003600CBC2BF0062406000D2
:101A20000004E0006000320050418000E10F5000EF
:101A300005003A000000EB00D04088000000EB00F9
:101A4000E0418800CDC2A8000000EB0050418800B2
:101A500010C0B3003AE8B70053003700CBC2BF0054
:101A6000624060000004E0000F003200504180003E
:101A7000E10F500009003A000040EB003AE8B700DF
:101A80000000EB00D04088000000EB00E04188003F
:101A9000CDC2A80010002000804188000000EB00AB
:101AA000504188000200370010002000504188009B
:101AB000E1418000F0408000808F500008003E002F
:101AC00080418000E10F500037003A000000EB0039
:101AD0005041880010C0B3003AE8B7003200370028
:101AE000CDC2A9000000EB00804188000000EB009F
:101AF000E04188000040EB003AE8B7002A003700D8
:101B0000CBC2BF00624060000004E0001D00320054
:101B10000040EB005AE8B70070418000E10F500030
:101B200003003A00604180000000E8006041880046
:101B3000F04280007800B9008000780060418000A9
:101B4000808F500018003E0050418000E10F50008F
:101B500005003A000000EB00D04088000000EB00D8
:101B6000E0418800CDC2A8000000EB007041880071
:101B70000000EB005041880010C0B3003AE8B70005
:101B8000090037001000200050418800100020009C
:101B9000704188000040EB003AE8B7000000EB001D
:101BA00060418800CDC2A90010C0B30060E8B70052
:101BB0006FFE3700620800005600000002000000BF
:101BC0000100040000000000020004000006000004
:101BD00008000A00000C00000E00100000120000B7
:101BE00014001800001C000020003000004000001D
:101BF0004B00D00007E80300F401C8000096000085
:101C000064003200000A0000050005000006000024
:101C1000060007000008000007000800000200009E
:101C200001000400004B0000000000000000000064
:101C3000000000000008000062000000000000003A
:101C4000F827000004000000000000000000000071
:101C5000F03FB1000180B10006003500EE0309003D
:101C600000000000403FB1000180B100FBFF3D00DB
:101C70001000B000203FB0000200350000800900D5
:101C800000000000000006000000FE00FFFFFF0053
:101C9000FFFFFF00FFFFFF00FFFFFF00FFFFFF0050
:101CA000FFFFFF00FFFFFF00FFFFFF00FFFFFF0040
:101CB000FFFFFF00FFFFFF00FFFFFF00FFFFFF0030
:101CC000FFFFFF00FFFFFF00FFFFFF00FFFFFF0020
:0200000401F009
:10000000CF000000CF00000007000000000000004B
:100010006500000059000000F5000000C30000006A
:00000001FF
